:03000000020C00EF
:03000300021A03DB
:03000B00021A06D0
:03001300021A09C5
:03001B00021A0CBA
:03002300021A0FAF
:03002B00021A12A4
:03003300021A1599
:03003B00021A188E
:03004300021A1B83
:03004B00021A1E78
:03005300021A216D
:03005B00021A2462
:03006300021A2757
:03006B00021A2A4C
:03007300021A2D41
:03007B00021A3036
:03008300021A332B
:03008B00021A3620
:03009300021A3915
:03009B00021A3C0A
:0300A300021A3FFF
:100C0000787FE4F6D8FD9000007F007E20E4F0A31A
:0A0C1000DFFCDEFA758121020C55AD
:104BDF0041055C00C100C10141055D004105600058
:104BEF004105610041056200410563004105640014
:105784009004A1E0FEA3E0FF90049DE0FCA3E0FDF3
:10579400B50719ECB5061590049FE0FEA3E0FFEDF4
:0E57A400B50709ECB5060520C502D322C322C5
:0A598A00E4F5847588107589022287
:0D597D00E4F584759A4075F809759D302297
:101A1B00E4F58475BCF8F5BA75E88075840275BC7D
:051A2B00F975E88022BE
:0759BF00E4F58475D1032219
:1058FA0075840F75AD0175A4CF75A50175A6777569
:09590A00A77F75E10375E3C022DB
:10561100E4FFFE75840F758A8353A1DFF58475B7A6
:10562100B075840F43A120438901758D01758F01E8
:10563100758E040FBF00010EEF640F4E70F54389A4
:0956410002E58930E4FB759702D3
:01564A00223D
:0A59940075A88243E6F343E71222F0
:10585D0012598A12597D121A1B1259BF1258FA1277
:10586D005611125994AF84E4F58475D4808F840257
:02587D0055D400
:1041580075FFDE75FFAD12585DE4FFFE0FBF00016D
:104168000EBE03F8BFE9F512587F90055AEFF0121A
:1041780059131257B2D2AF12554B12587F90055BA4
:10418800EFF090055AE06F6008A3E090055AF0D26E
:104198000090055DE06008121A33E490055DF012A6
:1041A8005724EF60D590059AE0FFB40B02D201EFD7
:1041B8006431704490055AE0FF90059BE06F7038B9
:1041C80012578450FB90055AE0FF12594112578448
:1041D80050FB90059CE0FFA3E0FDA3E0FBA3E0906B
:1041E8000537F012185612578450FB90055AE0FF15
:1041F80012592C12578450FB90059AE06432703E95
:1042080090055AE0FF90059BE06F7032125784507A
:10421800FB90055AE0FF12594112578450FB900554
:104228009CE0FFA3E0FDA3E0FB1248161257845060
:10423800FB90055AE0FF12592C12578450FB900549
:104248009AE0642D703E90055AE0FF90059BE06F60
:10425800703212578450FB90055AE0FF12594112F0
:10426800578450FB90059CE0FFA3E0FDA3E0FB1200
:10427800507312578450FB90055AE0FF12592C12C4
:10428800578450FB90059AE0642E703E90055AE0E2
:10429800FF90059BE06F703212578450FB90055ACF
:1042A800E0FF12594112578450FB90059CE0FFA390
:1042B800E0FDA3E0FB124EBF12578450FB90055A55
:1042C800E0FF12592C12578450FB90059AE0FFB476
:1042D800140890055C7401F0C20EEFB41505E49063
:1042E800055CF090055CE0700302418290059AE05D
:1042F80014601E04600302418290059BE0FFC39492
:104308001E4003024182900520EFF01257B202418D
:104318008290059BE0FFC3941E40030241829005F2
:0943280020EFF0121A3302418269
:031A060002531672
:10531600C0E0C0F0C083C082C0D075D000C000C05D
:1053260001C002C003C004C005C006C00775D30093
:10533600900562E014601514601714601914601B60
:1053460014601D2405701C1259DF8017124331802A
:105356001212599E800D123F2B8008124F9E800319
:10536600125956900562E004F0C3648094864002A8
:10537600E4F0D007D006D005D004D003D002D00187
:0D538600D000D0D0D082D083D0F0D0E03263
:10595600900564E0700312155D1259C6900564E067
:045966006401F022C6
:104BFF00C104C1054104F0804104F1804204F20078
:104C0F00004304FA0000004304FD000000430500C8
:104C1F00000000430503000000410506004104EDBC
:014C2F000183
:10587F00E5B0A2E29202E5B0A2E392033002093052
:10588F0003037F56227F57223003037F58227F590D
:01589F0022E6
:10155D009004F0E0A3F0E5B054029004F0F0A3E0A5
:10156D00FD9004F0E0FE6D9004E6F0EE7025ED6068
:10157D0005E4900506F0900506E004F0E0D394D064
:10158D00403F20050A90055AE0FF7D051258A0D274
:10159D0005802E9004F1E07028900506E0C394D0EC
:1015AD00501D30010990055CE06401F0801190053B
:1015BD005CE0600B90055D7401F0E490055CF0C299
:1015CD0005E49005C0F09005C0E0FFD364809482DF
:1015DD004003021702E0FEFD3395E0FC74FA2DF591
:1015ED008274043CF583E0FB74FD2DF58274043C9C
:1015FD00F583EBF0EE2404FE7401A806088002C307
:10160D0033D8FC55A0FEEFFD3395E0FC74FA2DF5B3
:10161D008274043CF583EEF09004EDE0601874FAEA
:10162D002DF58274043CF583E0FF74FD2DF5827475
:10163D00043CF583EFF09005C0E0FFFD3395E0FC31
:10164D0074FD2DF58274043CF583E0FE74FA2DF5DE
:10165D008274043CF583E06EFEEF3395E0FC74E795
:10166D002DF58274043CF583EEF074FA2DF5827439
:10167D00043CF583E0704274FD2DF58274043CF555
:10168D0083E06007E49004F2F0A3F09004F3E0042B
:10169D00F070069004F2E004F0D39004F3E094F0BF
:1016AD009004F2E0940040449004EFE0700312596E
:1016BD00B79004EF7401F080339005C0E0FFFD3367
:1016CD0095E0FC74FD2DF58274043CF583E0701CEF
:1016DD00C39004F3E094C09004F2E094005008EF3E
:1016ED003395E0FE12580AE49004EFF09005C0E047
:1016FD0004F00215D39005C07402F09005C0E0FF10
:10170D00C364809480500302184DE0FEFD3395E0D4
:10171D00FC74002DF58274053CF583E0FB74032DFC
:10172D00F58274053CF583EBF0EE2404FE7401A8FC
:10173D0006088002C333D8FC55B0FEEFFD3395E0AB
:10174D00FC74002DF58274053CF583EEF09004EDEC
:10175D00E0601874002DF58274053CF583E0FF748C
:10176D00032DF58274053CF583EFF09005C0E0FF85
:10177D00FD3395E0FC74032DF58274053CF583E093
:10178D00FE74002DF58274053CF583E06EFEEF339B
:10179D0095E0FC74EA2DF58274043CF583EEF0744B
:1017AD00002DF58274053CF583E0704E74032DF524
:1017BD008274053CF583E0601E9005C0E0FF339513
:1017CD00E0FEEF25E0FFEE33FE74F42FF582740496
:1017DD003EF583E4F0A3F09005C0E0FF3395E0FE05
:1017ED00EF25E0FFEE33FE74F42FF58274043EF521
:1017FD0083E475F001120FF5803D74032DF58274AD
:10180D00053CF583E070309005C0E0FD3395E0FCBC
:10181D00ED25E0FFEC33FE74F42FF58274043EF5F4
:10182D0083E0FEA3E0C394C0EE9400500AAF05AE72
:10183D00041256841258C09005C0E014F002170827
:08184D009004EDE06002E4F0FC
:011855002270
:1054B9009005A5E584F0A2AF920AAF01AE027C0087
:1054C900E4FDA31210949005A8E0FEA3E0780AA6D3
:1054D9000608F6E4F584C2AF43B701438F02438F50
:1054E9000118E6FE08E6F5828E83E4F053B7FEF56F
:0B54F9008FA20A92AF9005A5E0F58499
:015504002284
:05545D00900587EDF051
:10546200A3E584F0A2AF920BAF01AE027C00E4FD93
:10547200A3121094900587E0FFFD3395E0FCEDF454
:105482004C602990058BE0FCA3E0780CA60408F69A
:10549200E4F584C2AF43B701758F0118E6FC08E654
:1054A200F5828C83EFF053B7FEE4F58FA20B92AF37
:0654B200900588E0F5847E
:0154B80022D1
:1053930090058DEEF0A3EFF0A3ECF0A3EDF0A3EAFC
:1053A300F0A3EBF0900591E07002A3E06046900556
:1053B3008DE0FEA3E0AA06F97B01A3E0FEA3E0F5DE
:1053C300828E83E0FD12545D900592E024FFF090FD
:1053D3000591E034FFF0900590E004F0700690052D
:1053E3008FE004F090058EE004F070B890058DE036
:0553F30004F080B0226F
:0859A700E4900400F0A3F022DB
:10583400900400E0FEA3E0AA06F97B011254B9909B
:105844000400E0FEA3E0FF7C007D001B7A041253F9
:0958540093E4900400F0A3F0229B
:0D51EE0090057BEDF0900579EEF0A3EFF059
:1051FB00EE54FCFE900400E0FCA3E0FD7002EE6CAC
:10520B006059ED4C6003125834900579E0FEEE5472
:10521B00FCFE7F00900400F0A3EFF090057CEEF015
:10522B00A3EFF0A37400F0A37400F07FFF7E039054
:10523B00057CE475F00112100B85F082F583E49385
:10524B00FD90057EE475F00112100B85F082F5835D
:10525B00EDF0EF1F70011EEF4E70D490057BE0FF59
:10526B00900579E0FCA3E0FDEC5403FC74002DF5F4
:08527B008274003CF583EFF0A2
:015283002208
:10550500900593EEF0A3EFF0A3ECF0A3EDF0A3EA82
:10551500F0A3EBF090059774FFF5F012100B45F032
:105525006023900593E475F00112100BAFF0FE9027
:105535000595E475F00112100B85F082F583E0FD09
:065545001251EE80CF229E
:1058A0009005B6EFF0A3EDF07F0A1251459005B6D2
:1058B000E0FF1251459005B7E0FF125145021A0969
:0859AF007F02125145021A09A2
:065724001259CDEF6027D1
:10572A009005B87405F0A37499F01256BD9005B8A7
:10573A00E475F00112100B85F082F583EFF012592F
:07574A00D3EF70E67F01229E
:035751007F0022B4
:10592C009005C1EFF07F2F1251459005C1E0FF1299
:05593C005145021A09AB
:105941009005C2EFF07F301251459005C2E0FF1281
:055951005145021A0996
:104C30004105200043052100000041052400C10E6C
:105284001259A7E49005C3F09005C3E0FFC3940648
:105294005018EF25E02425F582E43405F583E4F085
:1052A400A3F09005C3E004F080DEE49005C3F09021
:1052B40005C3E0FFD39402502074312FF582E43407
:1052C40005F583E4F074212FF582E43405F583E4D5
:1052D400F09005C3E004F080D6E4900524F0900536
:1052E400C3F09005C3E0FFC3941E502375F00FEF85
:1052F400A42401F582E5F03480AF82FE7C057D258F
:105304007B0F7A001255059005C3E004F080D302A8
:0253140058340B
:105754009005BA7401F0E4A3F01259A77E807F008B
:105764007C057DBA7B017A001255057E817FC37C5E
:10577400057DBB7B017A0012550512583402528410
:1058C00030010F200E0C90055CE060061259AFD23B
:0E58D0000E2220010890055CE0700204F02218
:105913009081C3E493600C908000E493640160037E
:09592300125754E4900520F02213
:1057B200A2AF920CC2AF900520E075F00FA42401B5
:1057C200F9748035F0FA7BFF78257C057D017E0037
:0B57D2007F0F120FCFC20EA20C92AF8F
:0157DD0022A9
:1056F300A2AF920DC2AF1259A7900520E075F00F2B
:10570300A42401F582E5F03480AF82FE7C057D257B
:105713007B0F7A00125505125834C20EA20D92AFB8
:015723002263
:061A33001256F3C20E2260
:0A185600900535EDF0900534EFF039
:10186000D39B5003021934E024FFFEE434FF9005BB
:1018700039F0A3CEF0EB14900538F0900535E02454
:10188000FFFFE434FFFE900539E0FCA3E0FDD39FA9
:10189000EE6480F8EC6480984003021A05908001A1
:1018A00075F00FED1210D1EC75F00FA42583AF8207
:1018B000900540F0A3EFF0900538E075F00FA424F8
:1018C00001F9748035F0FA90053D74FFF0A3EAF059
:1018D000A3E9F0E490053BF0A3F090053DA3E47587
:1018E000F00112100BFEAFF0900540E475F001120C
:1018F000100B85F082F583E493FD1251EE90053CC8
:10190000E004F0700690053BE004F0C390053CE075
:10191000940F90053BE0940040C012583490053A73
:10192000E004F07006900539E004F0900538E0041A
:10193000F002187B900535E024FFFEE434FF9005AB
:1019400039F0A3CEF0900537E014A3F0900534E011
:1019500024FFFFE434FFFE900539E0FCA3E0FDC363
:101960009FEE6480F8EC6480985003021A05908022
:101970000175F00FED1210D1EC75F00FA42583AFB7
:1019800082900540F0A3EFF0900538E075F00FA4C9
:101990002401F9748035F0FA90053D74FFF0A3EA54
:1019A000F0A3E9F0E490053BF0A3F090053DA3E43B
:1019B00075F00112100BFEAFF0900540E475F001D8
:1019C00012100B85F082F583E493FD1251EE900521
:1019D0003CE004F0700690053BE004F0C390053C49
:1019E000E0940F90053BE0940040C01258349005FD
:1019F0003AE024FFF0900539E034FFF0900538E03C
:051A000014F002194C76
:011A050022BE
:05481600900507EDF024
:10481B00EF1490051CF0EB14A3F0900507E014FFC8
:10482B0090051CE0D39F4003024975A3E075F00F80
:10483B00A42401F582E5F03480AF82FEE490051EDE
:10484B00F0A3F090051EE0FCA3E0FDC3940FEC94E5
:10485B0000502B0FEFAA0670010E14F5828A83E429
:10486B0093FB740D2DF582E43405F583EBF0900585
:10487B001FE004F070CD90051EE004F080C590059C
:10488B001DE075F00FA42401F9748035F0FA900542
:10489B000874FFF0A3EAF0A3E9F090051CE075F0B3
:1048AB000FA42401F582E5F03480AF8290050BF064
:1048BB00A3EFF0E490051EF0A3F0900508A3E475B8
:1048CB00F00112100BFEAFF090050BE475F0011226
:1048DB00100B85F082F583E493FD1251EE90051FCA
:1048EB00E004F0700690051EE004F0C390051FE095
:1048FB00940F90051EE0940040C090051CE075F0ED
:10490B000FA42401F9748035F0FA90050874FFF0B8
:10491B00A3EAF0A3E9F0E490051EF0A3F090051EC6
:10492B00E0FCA3E0FDC3940FEC9400502D90050820
:10493B00A3E475F00112100BFEAFF0740D2DF58290
:10494B00E43405F583E0FD1251EE90051FE004F011
:10495B0070CB90051EE004F080C312583490051CF8
:0A496B00E004F0A3E004F002482588
:01497500221F
:074EBF00900565EBF0AC0764
:104EC600A2AFE433A3F0A3E584F0C2AFE4F584AF68
:104ED60005A3F0A3EFF0E07F00FE900568F0A3EFD6
:104EE600F0AD04EDFF900568EEF0A3EFF09005201D
:104EF600740FF01259A7900520E075F00FA4240155
:104F0600F9748035F0FA90056C74FFF0A3EAF0A30B
:104F1600E9F0E490056AF0A3F0900568E0FCA3E0F0
:104F2600FFECFD900565E0FBE49005ADF0D20612BE
:104F36004DDF90056FEFF0FD90056CA3E475F00171
:104F460012100BFEAFF01251EE900569E004F070FE
:104F560006900568E004F090056BE004F07006909A
:104F6600056AE004F0C390056BE0940F90056AE0D3
:104F7600940040A5125834900520E004F0E0C39454
:104F86001E5003024EF91255D4900567E0F5849041
:074F96000566E024FF92AF65
:014F9D0022F1
:07507300900570EBF0AC07A3
:10507A00A2AFE433A3F0A3E584F0C2AFE4F584AFB2
:10508A0005900575F0A3EFF0E07F00FE900575F03E
:10509A00A3EFF0AD04EDFF900575EEF0A3EFF090ED
:1050AA000520740FF0900520E0FFC3941E507A7516
:1050BA00F00FEFA42401F582E5F03480AF82900569
:1050CA0077F0A3EFF0E4900573F0A3F0900575E094
:1050DA00FCA3E0FFECFD900570E0FB900577E4751A
:1050EA00F00112100B85F082F583E4939005ADF080
:1050FA00C206124DDF900576E004F0700690057541
:10510A00E004F0900574E004F07006900573E00482
:10511A00F0C3900574E0940F900573E0940040ACDE
:10512A00900520E004F00250AF1255D4900572E0C9
:0A513A00F584900571E024FF92AFA8
:015144002248
:074DDF009005AAEFF0A90501
:104DE600C20720C3FD20C5FAC2C4D2C5E4FFFD3008
:104DF600C3FD30C3FDE5C154F8FC64086004ECB49F
:104E06001013EFB40105EB44018003EB54FEF5C229
:104E16007D01024EADECB4180B89C27D02C2C4C23C
:104E2600C5024EADECB420028045EC6428703CED22
:104E3600B4020E9005AAE0F5C27D03C2C5C2C480C5
:104E460066EDB4031B300608D2C57F01C2C4805785
:104E56009005ADE0F5C2C2C57D04E4FFC2C480473B
:104E6600ED64047042D2C47D05803CECB4300AD2B5
:104E7600C4D2C57D08E4FF802EECB438028024EC51
:104E8600B44006C2C2C2C5801EECB448028014EC0F
:104E9600B450028004ECB4580AD2C47D07AEC2C234
:104EA600C28004D2C4D2C5C2C3ED64076008ED64F3
:084EB600056003024DF8AF0690
:014EBE0022D1
:0A4C40004104B7004104B800C109A7
:1058DE00AF84E4F584C2C343E60243F60275C30106
:0B58EE0075C04475CF8F43C3018F8449
:0158F900228C
:1055D4007E047F89900487EEF0A3EFF0900485EEBB
:1055E400F0A3EFF0900483EEF0A3EFF07E047FA32A
:1055F4009004A1EEF0A3EFF090049FEEF0A3EFF07F
:0D56040090049DEEF0A3EFF0C2080258DE06
:10564B00900485E475F00112100B85F082F583EF61
:10565B00F0900485E475F00112100B85F082F58350
:10566B00EDF0900485E0B4040FA3E0B49D0A900420
:09567B00857404F0A37489F02287
:0D1A0900AF84E4F584C208C2C4D2C58F8446
:011A160022AD
:10514500200855D20890049FE475F00112100B85D4
:10515500F082F58374FFF07C047DB790049FE0B581
:10516500040FA3E0B5050A90049F7404F0A374A38B
:10517500F090049FE475F00112100B85F082F58321
:10518500E4F090049FE0B5040FA3E0B5050A900490
:105195009F7404F0A374A3F090049FE475F00112CA
:1051A500100B85F082F583E4F090049FE0B4040FC2
:1051B500A3E0B4B70A90049F7404F0A374A3F0901D
:1051C500049FE475F00112100B85F082F583EFF072
:1051D50090049FE0B4040FA3E0B4B70A90049F7451
:0951E50004F0A374A3F07F012281
:1057DE00900487E0FCA3E0FD900483E0B50408A3E9
:1057EE00E0B505037F0022900487E0FCA3E0F5827C
:0C57FE008C83E0B507037F01227F0022AE
:1056BD00900488E004F07006900487E004F09004F4
:1056CD0087E475F00112100B85F082F583E0FF90F1
:1056DD000487E0B4040FA3E0B49D0A90048774041A
:0556ED00F0A37489F038
:0156F2002295
:0659CD007FFF1257DE22ED
:0659D300E4FF1257DE2282
:031A1800023CF29B
:103CF200C0E0C0F0C083C082C0D075D000C000C098
:103D020004C005C006C007E5C154F81210DD3EE745
:103D1200003D4D083D4D103D9B183DE7203DF428E8
:103D22003E7F303E8B383E9C503E9C583EAF603EBC
:103D32009E683EAF703E9E783E9C803EBE883E9C12
:103D4200903EBE983ECFA000003F14C2C590049E94
:103D5200E004F0700690049DE004F07E047FB790CA
:103D6200049DE0B5060FA3E0B5070A90049D740414
:103D7200F0A374A3F090049DE475F00112100B857A
:103D8200F082F583E0F5C290049DE06E7003A3E03B
:103D92006F6003023F14023E7290049EE004F070D2
:103DA2000690049DE004F07E047FB790049DE0B588
:103DB200060FA3E0B5070A90049D7404F0A374A350
:103DC200F090049DE475F00112100B85F082F583EA
:103DD200E0F5C290049DE06E7003A3E06F60030201
:103DE2003F14023E729004A1E0FFA3E090049DCF35
:103DF200801B90049FE0FEA3E0FF90049DE0FCA3E3
:103E0200E0FDB50713ECB5060F9004A1EEF0A3EFA9
:103E1200F0C2C5D2C4023F148D828C83E0B4FF0786
:103E2200C2C4D2C5023F1490049EE004F070069012
:103E3200049DE004F07E047FB790049DE0B5060F78
:103E4200A3E0B5070A90049D7404F0A374A3F09054
:103E5200049DE475F00112100B85F082F583E0F504
:103E6200C290049DE06E7003A3E06F6003023F14F2
:103E720090049D7404F0A374A3F0023F149004A173
:103E8200E0FFA3E090049D803B9004A1E0FFA3E04B
:103E920090049DCFF0A3EFF0807880179004A1E00A
:103EA200FFA3E090049DCFF0A3EFF0D209ADC27F53
:103EB200FF8004ADC2E4FF12564B8056900483E0AB
:103EC200FFA3E0A3CFF0A3EFF0D2C4804590048516
:103ED200E0FFA3E0900483CFF0A3EFF0300933D2E8
:103EE200C5C209802D9004A1E0FEA3E0FF90049DCD
:103EF200EEF0A3EFF0900483E0FDA3E0A3CDF0A3E6
:103F0200EDF0D2C490049FE06E7003A3E06F6002F4
:103F1200D2C5C2C3D007D006D005D004D000D0D0BD
:093F2200D082D083D0F0D0E0324F
:1012020090FFFF121103EDF090FFFF121103EFF0B8
:0612120090FFEE12110333
:10121800850883850982E4F0A3F090001212112753
:10122800E025E02442F582E43405F583E0FEA3E0FE
:10123800FFFBAA06E4F9F8900012121127E025E056
:101248002403F582E43404F583E0FEA3E0FFC3EF52
:101258009BFFEE9AFEE499FDE498FC8508838509D6
:1012680082A3A3121094E47F40FEFDFC85088385C9
:101278000982A3A3E0F8A3E0F9A3E0FAA3E0FBC383
:1012880012107E400B850883850982E4F0A304F0E0
:1012980074FF7FC0FEFDFC850883850982A3A3E057
:1012A800F8A3E0F9A3E0FAA3E0FBD312107E500BF9
:1012B80085088385098274FFF0A3F0850883850972
:1012C80082E0FEA3E0FF4E7003021557EFF47002B0
:0712D800EEF460030213E4D1
:1012DF00900012121127E025E02442F582E4340534
:1012EF00F583E0FEA3E0FFE4FCFD90000E12112752
:1012FF00121094E47F01FEFDFC90000E121127E006
:10130F00F8A3E0F9A3E0FAA3E0FBC312107E500D9F
:10131F0090000E1211271210A00000000190001271
:10132F00121127E025E02425F582E43405F583E04A
:10133F00FEA3E0FFE4FCFD7BFF7A0FF9F81210210A
:10134F0090000E121127E0F8A3E0F9A3E0FAA3E052
:10135F00FB12559090000612112712109490001254
:10136F00121127E025E02403F582E43404F583E02D
:10137F00FEA3E0FFE4FCFD900006121127E0F8A3A6
:10138F00E0F9A3E0FAA3E0FB12102190000A12117A
:10139F0027121094E47BFF7A0FF9F890000A1211CC
:1013AF0027E0FCA3E0FDA3E0FEA3E0FF1255909021
:1013BF000012121127E025E02425F582E43405F50B
:1013CF0083EEF0A3EFF0900013121127E0700302E9
:0213DF00152EC9
:1013E10002152B850883850982E0FEA3E064014E86
:0513F100600302152E4F
:1013F600900012121127E025E02425F582E4340539
:10140600F583E0FEA3E0FBC374FF9BFF740F9EFE13
:10141600E49400FDE49400FCE47BFF7A0FF9F812F3
:10142600102190000612112712109490001212112A
:1014360027E025E02442F582E43405F583E0FEA3A7
:10144600E0FBC374FF9BFF740F9EFEE49400FDE473
:101456009400FC90000A121127121094E47F01FEFA
:10146600FDFC90000A121127E0F8A3E0F9A3E0FAC8
:10147600A3E0FBC312107E500D90000A1211271232
:1014860010A000000001900006121127C083C08240
:10149600E0FCA3E0FDA3E0FEA3E0FF90000A12112A
:1014A60027E0F8A3E0F9A3E0FAA3E0FB125590D0F9
:1014B60082D083121094900012121127E025E024A6
:1014C60003F582E43404F583E0FEA3E0FBC374FF76
:1014D6009BFF740F9EFEE49400FDE49400FC9000D4
:1014E60006121127E0F8A3E0F9A3E0FAA3E0FB1245
:1014F6001021E47BFF7A0FF9F8125590C374FF9F11
:10150600FF740F9EFE900012121127E025E024259D
:10151600F582E43405F583EEF0A3EFF090001312A4
:081526001127E060031258C018
:10152E00900012121127E0FF25E02403F582E43427
:10153E0004F583E0FCA3E0FDEF25E02442F582E410
:09154E003405F583ECF0A3EDF087
:06155700900014021103D4
:0659D90030313234353696
:104F9E00E4FDFCC3ED9403EC648094805023ED2576
:104FAE00E0FFEC33FE744E2FF58274053EF583A3BD
:104FBE00E0C4F8540FC868FF0582D58202158380BD
:104FCE002CC3ED9406EC64809480502FED25E0FF09
:104FDE00EC33FE74472FF58274043EF583A3E0C4D0
:104FEE00F8540FC868FF0582D5820215831582E03A
:104FFE00C454F0489005BCF0A3EFF074D92DF5829F
:10500E0074593CF583E493FFE4F584C2FA8F9B3028
:10501E00FFFDC2FFE4FFFE0FBF00010EEF64324E34
:10502E0070F59005BCE0F59B30FFFDC2FFE4FEFF7E
:10503E000FBF00010EEF64324E70F59005BDE0F526
:10504E009B30FFFDC2FFE4FEFF0FBF00010EEF64B9
:10505E00324E70F5D2FA0DBD00010CED64064C60B7
:04506E0003024FA149
:01507200221B
:104C4A004304BF0002044304C204000C4304C50623
:104C5A00020E4304C805010D4304CB07030F4304A6
:104C6A00CE090A0B4304D10B0F074304D40A0E06DC
:104C7A004304D7090D054304DA080C044304DD0391
:104C8A0002014204E000004204E20000C10F4304B2
:0F4C9A00B91919194304BC1010104204E40000AA
:103A3C009004E0E0FFA3E09005AECFF0A3EFF0E43C
:103A4C009004E0F0A3F0FDED25E0244DF582E43484
:103A5C0004F583E0FEC3EE940F401F74C22DF58273
:103A6C00E43404F583E0FF74017E00A807088005A8
:103A7C00C333CE33CED8F9023B26ED25E0244DF5E9
:103A8C0082E43404F583E0FEA3E0C394FFEE9409D2
:103A9C00401E74C82DF582E43404F583E0FF7401F4
:103AAC007E00A807088005C333CE33CED8F9806AD0
:103ABC00ED25E0244DF582E43404F583E0FEA3E02B
:103ACC00C394FFEE9406401E74C52DF582E43404B5
:103ADC00F583E0FF74017E00A807088005C333CE90
:103AEC0033CED8F98034ED25E0244DF582E434044E
:103AFC00F583E0FEA3E0C394FFEE9403402774CB60
:103B0C002DF582E43404F583E0FF74017E00A807F0
:103B1C00088005C333CE33CED8F9FF9004E0E04ED5
:103B2C00F0A3E04FF0ED25E02454F582E43405F5E4
:103B3C0083E0FEA3E064024E7042EDFFC374029F6B
:103B4C00FFE49400FE74CE2FF58274043EF583E0FE
:103B5C00FF74017E00A807088005C333CE33CED88E
:103B6C00F9FF9004E0E04EF0A3E04FF074B92DF5AE
:103B7C0082E43404F5837419F0023C3EED25E02414
:103B8C0054F582E43405F583E0FEA3E064014E6055
:103B9C0003023C3E74B92DF582E43404F583E060F5
:103BAC004374B92DF582E43404F583E014F06034E9
:103BBC00EDFFC374029FFFE49400FE74CE2FF582D8
:103BCC0074043EF583E0FF74017E00A807088005AD
:103BDC00C333CE33CED8F9FF9004E0E04EF0A3E02F
:103BEC004FF0804E74BC2DF582E43404F583E01460
:103BFC00F0703FEDFFC374029FFFE49400FE74CE9F
:103C0C002FF58274043EF583E0FF74017E00A80753
:103C1C00088005C333CE33CED8F9FF9004E0E04ED4
:103C2C00F0A3E04FF074BC2DF582E43404F58374FA
:0D3C3C0010F00DED64036003023A53C2B0B6
:103C49009005B0E4F0A37410F09005B074FFF5F09E
:0E3C590012100BFED3E5F09400EE940050EB39
:103C6700E4FD9004E0E0FEA3E0A805088005CEC3CC
:0A3C770013CE13D8F9139286C2870A
:103C81009005B0E4F0A37410F09005B074FFF5F066
:0E3C910012100BFED3E5F09400EE940050EB01
:023C9F00D287CA
:103CA1009005B0E4F0A37410F09005B074FFF5F046
:0E3CB10012100BFED3E5F09400EE940050EBE1
:0B3CBF00ED64076004EDB40F20D2B0EC
:103CCA009005B0E4F0A37410F09005B074FFF5F01D
:0E3CDA0012100BFED3E5F09400EE940050EBB8
:093CE8000DED64106003023C695B
:013CF10022B0
:1044D600E49004E2F0A3F0FD74212DF582E43405A6
:1044E600F583E01460251460402402706374D12DB6
:1044F600F582E43404F583E0FF74017E00A8070822
:104506008005C333CE33CED8F9803A74D42DF582E4
:10451600E43404F583E0FF74017E00A807088005F3
:10452600C333CE33CED8F9801C74D72DF582E4344C
:1045360004F583E0FF74017E00A807088005C333F5
:10454600CE33CED8F9FF9004E2E04EF0A3E04FF070
:10455600900524E0602774DA2DF582E43404F583AF
:10456600E0FF74017E00A807088005C333CE33CE72
:10457600D8F9FF9004E2E04EF0A3E04FF074312D3D
:10458600F582E43405F583E0602774DD2DF582E4D9
:104596003404F583E0FF74017E00A807088005C394
:1045A60033CE33CED8F9FF9004E2E04EF0A3E04FCD
:1045B600F090055CE060079004E3E04401F00DED47
:0945C600640360030244DEC2A29A
:1045CF009005BEE4F0A37410F09005BE74FFF5F0F3
:0E45DF0012100BFED3E5F09400EE940050EBAA
:1045ED00E4FD9004E2E0FEA3E0A805088005CEC33B
:0A45FD0013CE13D8F91392A0C2A147
:104607009005BEE4F0A37410F09005BE74FFF5F0BA
:0E46170012100BFED3E5F09400EE940050EB71
:02462500D2A120
:104627009005BEE4F0A37410F09005BE74FFF5F09A
:0E46370012100BFED3E5F09400EE940050EB51
:0B464500ED64076004EDB40F20D2A26A
:104650009005BEE4F0A37410F09005BE74FFF5F071
:0E46600012100BFED3E5F09400EE940050EB28
:09466E000DED641060030245EF3C
:014677002220
:0759C600123A3C1244D62204
:10580A0074212FF58274053EF583E004F074212F8C
:10581A00F58274053EF583E0D39402400C74212F7F
:0A582A00F58274053EF583E4F022D8
:10568400C374029FFDE49EFC74312DF58274053CC5
:10569400F583E004F074312DF58274053CF583E064
:1056A400D39401401374029FFFE49EFE74312FF5DE
:0956B4008274053EF583E4F02246
:0859B700900524E06401F022D8
:104CA90041043E0041043F004104400041044100E9
:104CB9004A04420000000200040006000741040201
:014CC90001E9
:0459DF0043E8102267
:09599E00758402D2ECE4F58422C8
:031A3000024CEA7B
:104CEA00C0E0C083C082C0D075D000C004C005C077
:104CFA0006C00753E8DFAFBFEFFEADBE7C00E42D70
:104D0A00FFEC3E90043BF0A3EFF090043BE0FCA3E1
:104D1A00E0FD90043EE0FF3395E0FEEF25E0FFEE74
:104D2A0033FE74422FF58274043EF583A3E025E036
:104D3A00FF0582D5820215831582E033FE740F2F98
:104D4A00F58274043EF583ECF0A3EDF090043EE0A6
:104D5A0004F0C364809485404DE4F090040FE0FFB2
:104D6A00A3E090042FCFF0A3EFF0900413E0FFA389
:104D7A00E0900431CFF0A3EFF0900417E0FFA3E036
:104D8A00900433CFF0A3EFF090041BE0FFA3E09070
:104D9A000437CFF0A3EFF090041DE0FFA3E09004E6
:104DAA0039CFF0A3EFF090043EE0FF3395E0FEEF39
:104DBA0025E0FFEE33FE74422FF58274043EF5833C
:104DCA00A3E0F5BBD007D006D005D004D0D0D0825E
:054DDA00D083D0E0329F
:031A3900024678EA
:10467800C0E0C0F0C083C082C0D075D000C000C008
:0D46880001C002C003C004C005C006C00789
:1046950075840253E8DFC2ED90043DE5BEF0E07598
:1046A500F010A4FD90043FE0FF3395E0FEEF25E018
:1046B500FFEE33FE741F2FF58274043EF583E5F09B
:1046C500F0A3EDF090043FE004F0C36480948850BB
:1046D500030247F27401F090042DE0FFA3E090047B
:1046E50035CFF0A3EFF0900421E0FFA3E0900403A1
:1046F500CFF0A3EFF0900423E0FFA3E0900405CFF3
:10470500F0A3EFF0900425E0FFA3E0900407CFF0BD
:10471500A3EFF0900427E0FFA3E0900409CFF0A3F6
:10472500EFF0900429E0FFA3E090040BCFF0A3EF96
:10473500F090042BE0FFA3E090040DCFF0A3EFF081
:10474500900402E06041E4FDFCED25E0FFEC33FE62
:1047550074032FF58274043EF583E0FAA3E0FB743D
:10476500422FF58274053EF583EAF0A3EBF00DBD0B
:1047750000010CED64064C70D0900402E004F0E0FA
:10478500D3940A4002E4F0900402E070047D0180B5
:10479500027D007F00121202900402E070047D0188
:1047A50080027D007F01121202900402E070047DF8
:1047B5000180027D007F02121202900402E0700463
:1047C5007D0180027D007F03121202900402E070D9
:1047D500047D0180027D007F04121202900402E034
:1047E50070047D0180027D007F0512120290043F56
:0647F500E0F5BB75840035
:1047FB00D007D006D005D004D003D002D001D00012
:0B480B00D0D0D082D083D0F0D0E032BB
:101A3C0000C800C700C700C700C700C700C700C662
:101A4C0000C600C600C600C600C600C600C500C55C
:101A5C0000C500C500C500C500C500C400C400C455
:101A6C0000C400C400C400C400C300C300C300C34E
:101A7C0000C300C300C300C200C200C200C200C247
:101A8C0000C200C100C100C100C100C100C100C141
:101A9C0000C000C000C000C000C000C000C000BF3B
:101AAC0000BF00BF00BF00BF00BF00BF00BE00BE34
:101ABC0000BE00BE00BE00BE00BE00BD00BD00BD2D
:101ACC0000BD00BD00BD00BD00BC00BC00BC00BC26
:101ADC0000BC00BC00BB00BB00BB00BB00BB00BB20
:101AEC0000BB00BA00BA00BA00BA00BA00BA00BA19
:101AFC0000B900B900B900B900B900B900B900B813
:101B0C0000B800B800B800B800B800B800B700B70B
:101B1C0000B700B700B700B700B600B600B600B605
:101B2C0000B600B600B600B500B500B500B500B5FE
:101B3C0000B500B500B400B400B400B400B400B4F7
:101B4C0000B400B300B300B300B300B300B300B3F0
:101B5C0000B200B200B200B200B200B200B200B1EA
:101B6C0000B100B100B100B100B100B000B000B0E4
:101B7C0000B000B000B000B000AF00AF00AF00AFDD
:101B8C0000AF00AF00AF00AE00AE00AE00AE00AED6
:101B9C0000AE00AE00AD00AD00AD00AD00AD00ADCF
:101BAC0000AD00AC00AC00AC00AC00AC00AC00ABC9
:101BBC0000AB00AB00AB00AB00AB00AB00AA00AAC3
:101BCC0000AA00AA00AA00AA00AA00A900A900A9BC
:101BDC0000A900A900A900A900A800A800A800A8B5
:101BEC0000A800A800A800A700A700A700A700A7AE
:101BFC0000A700A700A600A600A600A600A600A6A7
:101C0C0000A500A500A500A500A500A500A500A4A1
:101C1C0000A400A400A400A400A400A400A300A39A
:101C2C0000A300A300A300A300A300A200A200A293
:101C3C0000A200A200A200A200A100A100A100A18C
:101C4C0000A100A100A000A000A000A000A000A086
:101C5C0000A0009F009F009F009F009F009F009F7F
:101C6C00009E009E009E009E009E009E009E009D79
:101C7C00009D009D009D009D009D009D009C009C72
:101C8C00009C009C009C009C009C009B009B009B6B
:101C9C00009B009B009B009A009A009A009A009A65
:101CAC00009A009A0099009900990099009900995E
:101CBC000099009800980098009800980098009857
:101CCC000097009700970097009700970097009651
:101CDC00009600960096009600960096009500954A
:101CEC000095009500950095009400940094009444
:101CFC00009400940094009300930093009300933D
:101D0C000093009300920092009200920092009235
:101D1C00009200910091009100910091009100912E
:101D2C00009000900090009000900090008F008F29
:101D3C00008F008F008F008F008F008E008E008E22
:101D4C00008E008E008E008E008D008D008D008D1B
:101D5C00008D008D008D008C008C008C008C008C14
:101D6C00008C008C008B008B008B008B008B008B0D
:101D7C00008B008A008A008A008A008A008A008907
:101D8C000089008900890089008900890088008801
:101D9C0000880088008800880088008700870087FA
:101DAC0000870087008700870086008600860086F3
:101DBC0000860086008600850085008500850085EC
:101DCC0000850084008400840084008400840084E6
:101DDC0000830083008300830083008300830082E0
:101DEC0000820082008200820082008200810081D9
:101DFC0000810081008100810081008000800080D2
:101E0C000080008000800080007F007F007F007FCA
:101E1C00007F007F007E007E007E007E007E007EC4
:101E2C00007E007D007D007D007D007D007D007DBD
:101E3C00007C007C007C007C007C007C007C007BB7
:101E4C00007B007B007B007B007B007B007A007AB0
:101E5C00007A007A007A007A0079007900790079AA
:101E6C0000790079007900780078007800780078A3
:101E7C00007800780077007700770077007700779C
:101E8C000077007600760076007600760076007695
:101E9C00007500750075007500750075007500748F
:101EAC000074007400740074007400730073007389
:101EBC000073007300730073007200720072007282
:101ECC00007200720072007100710071007100717B
:101EDC000071007100700070007000700070007074
:101EEC000070006F006F006F006F006F006F006E6E
:101EFC00006E006E006E006E006E006E006D006D68
:101F0C00006D006D006D006D006D006C006C006C60
:101F1C00006C006C006C006C006B006B006B006B59
:101F2C00006B006B006B006A006A006A006A006A52
:101F3C00006A006A0069006900690069006900694B
:101F4C000068006800680068006800680068006746
:101F5C00006700670067006700670067006600663F
:101F6C000066006600660066006600650065006538
:101F7C000065006500650065006400640064006431
:101F8C00006400640064006300630063006300632A
:101F9C00006300630063006300630063006200621F
:101FAC000062006200620062006200620062006215
:101FBC00006200610061006100610061006100610C
:101FCC000061006100610061006100600060006000
:101FDC0000600060006000600060006000600060F5
:101FEC00005F005F005F005F005F005F005F005FED
:101FFC00005F005F005F005E005E005E005E005EE2
:10200C00005E005E005E005E005E005E005E005DD5
:10201C00005D005D005D005D005D005D005D005DCC
:10202C00005D005D005C005C005C005C005C005CC2
:10203C00005C005C005C005C005C005B005B005BB7
:10204C00005B005B005B005B005B005B005B005BAC
:10205C00005B005A005A005A005A005A005A005AA3
:10206C00005A005A005A005A005900590059005998
:10207C00005900590059005900590059005900598C
:10208C000058005800580058005800580058005884
:10209C000058005800580057005700570057005779
:1020AC00005700570057005700570057005600566E
:1020BC000056005600560056005600560056005664
:1020CC00005600560055005500550055005500555A
:1020DC00005500550055005500550054005400544F
:1020EC000054005400540054005400540054005444
:1020FC00005300530053005300530053005300533C
:10210C00005300530053005300520052005200522F
:10211C000052005200520052005200520052005124
:10212C00005100510051005100510051005100511B
:10213C000051005100500050005000500050005011
:10214C00005000500050005000500050004F004F05
:10215C00004F004F004F004F004F004F004F004FFB
:10216C00004F004E004E004E004E004E004E004EF2
:10217C00004E004E004E004E004E004D004D004DE6
:10218C00004D004D004D004D004D004D004D004DDB
:10219C00004C004C004C004C004C004C004C004CD3
:1021AC00004C004C004C004B004B004B004B004BC8
:1021BC00004B004B004B004B004B004B004B004ABC
:1021CC00004A004A004A004A004A004A004A004AB3
:1021DC00004A004A004900490049004900490049A9
:1021EC00004900490049004900490048004800489E
:1021FC000048004800480048004800480048004893
:10220C000048004700470047004700470047004789
:10221C00004700470047004700460046004600467E
:10222C000046004600460046004600460046004672
:10223C00004500450045004500450045004500456A
:10224C00004500450045004400440044004400445F
:10225C000044004400440044004400440043004354
:10226C00004300430043004300430043004300434A
:10227C000043004300420042004200420042004240
:10228C000042004200420042004200410041004135
:10229C00004100410041004100410041004100412A
:1022AC000040004000400040004000400040004022
:1022BC000040004000400040003F003F003F003F16
:1022CC00003F003F003F003F003F003F003F003E0B
:1022DC00003E003E003E003E003E003E003E003E02
:1022EC00003E003E003D003D003D003D003D003DF8
:1022FC00003D003D003D003D003D003D003C003CEC
:10230C00003C003C003C003C003C003C003C003CE1
:10231C00003C003B003B003B003B003B003B003BD8
:10232C00003B003B003B003B003B003A003A003ACC
:10233C00003A003A003A003A003A003A003A003AC1
:10234C0000390039003900390039003900390039B9
:10235C0000390039003900380038003800380038AE
:10236C0000380038003800380038003800380037A2
:10237C000037003700370037003700370037003799
:10238C00003700370036003600360036003600368F
:10239C000036003600360036003600350035003584
:1023AC000035003500350035003500350035003579
:1023BC000035003400340034003400340034003470
:1023CC000034003400340034003300330033003365
:1023DC00003300330033003300330033003300325A
:1023EC000032003200320032003200320032003251
:1023FC000032003200320031003100310031003146
:10240C00003100310031003100310031003000303A
:10241C000030003000300030003000300030003030
:10242C0000300030002F002F002F002F002F002F26
:10243C00002F002F002F002F002F002E002E002E1B
:10244C00002E002E002E002E002E002E002E002E10
:10245C00002D002D002D002D002D002D002D002D08
:10246C00002D002D002D002D002C002C002C002CFC
:10247C00002C002C002C002C002C002C002C002BF1
:10248C00002B002B002B002B002B002B002B002BE8
:10249C00002B002B002A002A002A002A002A002ADE
:1024AC00002A002A002A002A002A002A00290029D2
:1024BC0000290029002900290029002900290029C8
:1024CC0000290028002800280028002800280028BF
:1024DC0000280028002800280028002700270027B3
:1024EC0000270027002700270027002700270027A8
:1024FC000027002700270027002700270027002798
:10250C000027002700270027002700270027002787
:10251C000027002700270027002700270027002678
:10252C00002600260026002600260026002600266F
:10253C00002600260026002600260026002600265F
:10254C00002600260026002600260026002600264F
:10255C00002600260026002600260026002600263F
:10256C000026002500250025002500250025002536
:10257C000025002500250025002500250025002527
:10258C000025002500250025002500250025002517
:10259C000025002500250025002500250025002507
:1025AC0000250025002500240024002400240024FC
:1025BC0000240024002400240024002400240024EF
:1025CC0000240024002400240024002400240024DF
:1025DC0000240024002400240024002400240024CF
:1025EC0000240024002400240024002300230023C2
:1025FC0000230023002300230023002300230023B7
:10260C0000230023002300230023002300230023A6
:10261C000023002300230023002300230023002396
:10262C000023002300230023002300230023002287
:10263C00002200220022002200220022002200227E
:10264C00002200220022002200220022002200226E
:10265C00002200220022002200220022002200225E
:10266C00002200220022002200220022002200224E
:10267C000022002100210021002100210021002145
:10268C000021002100210021002100210021002136
:10269C000021002100210021002100210021002126
:1026AC000021002100210021002100210021002116
:1026BC00002100210021002000200020002000200B
:1026CC0000200020002000200020002000200020FE
:1026DC0000200020002000200020002000200020EE
:1026EC0000200020002000200020002000200020DE
:1026FC0000200020002000200020001F001F001FD1
:10270C00001F001F001F001F001F001F001F001FC5
:10271C00001F001F001F001F001F001F001F001FB5
:10272C00001F001F001F001F001F001F001F001FA5
:10273C00001F001F001F001F001F001F001F001E96
:10274C00001E001E001E001E001E001E001E001E8D
:10275C00001E001E001E001E001E001E001E001E7D
:10276C00001E001E001E001E001E001E001E001E6D
:10277C00001E001E001E001E001E001E001E001E5D
:10278C00001E001E001D001D001D001D001D001D53
:10279C00001D001D001D001D001D001D001D001D45
:1027AC00001D001D001D001D001D001D001D001D35
:1027BC00001D001D001D001D001D001D001D001D25
:1027CC00001D001D001D001D001C001C001C001C19
:1027DC00001C001C001C001C001C001C001C001C0D
:1027EC00001C001C001C001C001C001C001C001CFD
:1027FC00001C001C001C001C001C001C001C001CED
:10280C00001C001C001C001C001C001C001B001BDE
:10281C00001B001B001B001B001B001B001B001BD4
:10282C00001B001B001B001B001B001B001B001BC4
:10283C00001B001B001B001B001B001B001B001BB4
:10284C00001B001B001B001B001B001B001B001BA4
:10285C00001A001A001A001A001A001A001A001A9C
:10286C00001A001A001A001A001A001A001A001A8C
:10287C00001A001A001A001A001A001A001A001A7C
:10288C00001A001A001A001A001A001A001A001A6C
:10289C00001A001A00190019001900190019001962
:1028AC000019001900190019001900190019001954
:1028BC000019001900190019001900190019001944
:1028CC000019001900190019001900190019001934
:1028DC000019001900190019001800180018001828
:1028EC00001800180018001800180018001800181C
:1028FC00001800180018001800180018001800180C
:10290C0000180018001800180018001800180018FB
:10291C0000180018001800180018001800170017ED
:10292C0000170017001700170017001700170017E3
:10293C0000170017001700170017001700170017D3
:10294C0000170017001700170017001700170017C3
:10295C0000170017001700170017001700170017B3
:10296C0000160016001600160016001600160016AB
:10297C00001600160016001600160016001600169B
:10298C00001600160016001600160016001600168B
:10299C00001600160016001600160016001600167B
:1029AC000016001600150015001500150015001571
:1029BC000015001500150015001500150015001563
:1029CC000015001500150015001500150015001553
:1029DC000015001500150015001500150015001543
:1029EC000015001500150015001400140014001437
:1029FC00001400140014001400140014001400142B
:102A0C00001400140014001400140014001400141A
:102A1C00001400140014001400140014001400140A
:102A2C0000140014001400140014001400140013FB
:102A3C0000130013001300130013001300130013F2
:102A4C0000130013001300130013001300130013E2
:102A5C0000130013001300130013001300130013D2
:102A6C0000130013001300130013001300130013C2
:102A7C0000130013001300130013001300130013B2
:102A8C0000130013001300130013001300130013A2
:102A9C000013001300130013001300130013001392
:102AAC000013001300130013001300130013001382
:102ABC000013001300130012001200120012001277
:102ACC00001200120012001200120012001200126A
:102ADC00001200120012001200120012001200125A
:102AEC00001200120012001200120012001200124A
:102AFC00001200120012001200120012001200123A
:102B0C000012001200120012001200120012001229
:102B1C000012001200120012001200120012001219
:102B2C000012001200120012001200120012001209
:102B3C0000120012001200120012001200120011FA
:102B4C0000110011001100110011001100110011F1
:102B5C0000110011001100110011001100110011E1
:102B6C0000110011001100110011001100110011D1
:102B7C0000110011001100110011001100110011C1
:102B8C0000110011001100110011001100110011B1
:102B9C0000110011001100110011001100110011A1
:102BAC000011001100110011001100110011001191
:102BBC000011001100110011001100110011001181
:102BCC000011001100110010001000100010001076
:102BDC000010001000100010001000100010001069
:102BEC000010001000100010001000100010001059
:102BFC000010001000100010001000100010001049
:102C0C000010001000100010001000100010001038
:102C1C000010001000100010001000100010001028
:102C2C000010001000100010001000100010001018
:102C3C000010001000100010001000100010001008
:102C4C000010001000100010001000100010000FF9
:102C5C00000F000F000F000F000F000F000F000FF0
:102C6C00000F000F000F000F000F000F000F000FE0
:102C7C00000F000F000F000F000F000F000F000FD0
:102C8C00000F000F000F000F000F000F000F000FC0
:102C9C00000F000F000F000F000F000F000F000FB0
:102CAC00000F000F000F000F000F000F000F000FA0
:102CBC00000F000F000F000F000F000F000F000F90
:102CCC00000F000F000F000F000F000F000F000F80
:102CDC00000F000F000F000F000E000E000E000E74
:102CEC00000E000E000E000E000E000E000E000E68
:102CFC00000E000E000E000E000E000E000E000E58
:102D0C00000E000E000E000E000E000E000E000E47
:102D1C00000E000E000E000E000E000E000E000E37
:102D2C00000E000E000E000E000E000E000E000E27
:102D3C00000E000E000E000E000E000E000E000E17
:102D4C00000E000E000E000E000E000E000E000E07
:102D5C00000E000E000E000E000E000E000E000EF7
:102D6C00000D000D000D000D000D000D000D000DEF
:102D7C00000D000D000D000D000D000D000D000DDF
:102D8C00000D000D000D000D000D000D000D000DCF
:102D9C00000D000D000D000D000D000D000D000DBF
:102DAC00000D000D000D000D000D000D000D000DAF
:102DBC00000D000D000D000D000D000D000D000D9F
:102DCC00000D000D000D000D000D000D000D000D8F
:102DDC00000D000D000D000D000D000D000D000D7F
:102DEC00000D000D000D000D000C000C000C000C73
:102DFC00000C000C000C000C000C000C000C000C67
:102E0C00000C000C000C000C000C000C000C000C56
:102E1C00000C000C000C000C000C000C000C000C46
:102E2C00000C000C000C000C000C000C000C000C36
:102E3C00000C000C000C000C000C000C000C000C26
:102E4C00000C000C000C000C000C000C000C000C16
:102E5C00000C000C000C000C000C000C000C000C06
:102E6C00000C000C000C000C000C000C000C000CF6
:102E7C00000B000B000B000B000B000B000B000BEE
:102E8C00000B000B000B000B000B000B000B000BDE
:102E9C00000B000B000B000B000B000B000B000BCE
:102EAC00000B000B000B000B000B000B000B000BBE
:102EBC00000B000B000B000B000B000B000B000BAE
:102ECC00000B000B000B000B000B000B000B000B9E
:102EDC00000B000B000B000B000B000B000B000B8E
:102EEC00000B000B000B000B000B000B000B000B7E
:102EFC00000B000B000B000B000A000A000A000A72
:102F0C00000A000A000A000A000A000A000A000A65
:102F1C00000A000A000A000A000A000A000A000A55
:102F2C00000A000A000A000A000A000A000A000A45
:102F3C00000A000A000A000A000A000A000A000A35
:102F4C00000A000A000A000A000A000A000A000A25
:102F5C00000A000A000A000A000A000A000A000A15
:102F6C00000A000A000A000A000A000A000A000A05
:102F7C00000A000A000A000A000A000A000A000AF5
:102F8C00000A0009000900090009000900090009EC
:102F9C0000090009000900090009000900090009DD
:102FAC0000090009000900090009000900090009CD
:102FBC0000090009000900090009000900090009BD
:102FCC0000090009000900090009000900090009AD
:102FDC00000900090009000900090009000900099D
:102FEC00000900090009000900090009000900098D
:102FFC00000900090009000900090009000900097D
:10300C00000900090009000900090009000900096C
:10301C00000900090009000900090009000900095C
:10302C00000900090009000900090009000900094C
:10303C00000900090009000900090009000900093C
:10304C00000900090009000900090009000900092C
:10305C00000900090009000900090009000900091C
:10306C00000900090009000900090009000900090C
:10307C0000090009000900090009000900090009FC
:10308C0000090009000900090009000900090009EC
:10309C0000090008000800080008000800080008E3
:1030AC0000080008000800080008000800080008D4
:1030BC0000080008000800080008000800080008C4
:1030CC0000080008000800080008000800080008B4
:1030DC0000080008000800080008000800080008A4
:1030EC000008000800080008000800080008000894
:1030FC000008000800080008000800080008000884
:10310C000008000800080008000800080008000873
:10311C000008000800080008000800080008000863
:10312C000008000800080008000800080008000853
:10313C000008000800080008000800080008000843
:10314C000008000800080008000800080008000833
:10315C000008000800080008000800080008000823
:10316C000008000800080008000800080008000813
:10317C000008000800080008000800080008000803
:10318C0000080008000800080008000800080008F3
:10319C0000080008000800080008000800080008E3
:1031AC0000080007000700070007000700070007DA
:1031BC0000070007000700070007000700070007CB
:1031CC0000070007000700070007000700070007BB
:1031DC0000070007000700070007000700070007AB
:1031EC00000700070007000700070007000700079B
:1031FC00000700070007000700070007000700078B
:10320C00000700070007000700070007000700077A
:10321C00000700070007000700070007000700076A
:10322C00000700070007000700070007000700075A
:10323C00000700070007000700070007000700074A
:10324C00000700070007000700070007000700073A
:10325C00000700070007000700070007000700072A
:10326C00000700070007000700070007000700071A
:10327C00000700070007000700070007000700070A
:10328C0000070007000700070007000700070007FA
:10329C0000070007000700070007000700070007EA
:1032AC0000070007000700070007000700070007DA
:1032BC0000070007000600060006000600060006D0
:1032CC0000060006000600060006000600060006C2
:1032DC0000060006000600060006000600060006B2
:1032EC0000060006000600060006000600060006A2
:1032FC000006000600060006000600060006000692
:10330C000006000600060006000600060006000681
:10331C000006000600060006000600060006000671
:10332C000006000600060006000600060006000661
:10333C000006000600060006000600060006000651
:10334C000006000600060006000600060006000641
:10335C000006000600060006000600060006000631
:10336C000006000600060006000600060006000621
:10337C000006000600060006000600060006000611
:10338C000006000600060006000600060006000601
:10339C0000060006000600060006000600060006F1
:1033AC0000060006000600060006000600060006E1
:1033BC0000060006000600060006000600060006D1
:1033CC0000060006000500050005000500050005C7
:1033DC0000050005000500050005000500050005B9
:1033EC0000050005000500050005000500050005A9
:1033FC000005000500050005000500050005000599
:10340C000005000500050005000500050005000588
:10341C000005000500050005000500050005000578
:10342C000005000500050005000500050005000568
:10343C000005000500050005000500050005000558
:10344C000005000500050005000500050005000548
:10345C000005000500050005000500050005000538
:10346C000005000500050005000500050005000528
:10347C000005000500050005000500050005000518
:10348C000005000500050005000500050005000508
:10349C0000050005000500050005000500050005F8
:1034AC0000050005000500050005000500050005E8
:1034BC0000050005000500050005000500050005D8
:1034CC0000050005000500050005000500050005C8
:1034DC0000050005000500040004000400040004BD
:1034EC0000040004000400040004000400040004B0
:1034FC0000040004000400040004000400040004A0
:10350C00000400040004000400040004000400048F
:10351C00000400040004000400040004000400047F
:10352C00000400040004000400040004000400046F
:10353C00000400040004000400040004000400045F
:10354C00000400040004000400040004000400044F
:10355C00000400040004000400040004000400043F
:10356C00000400040004000400040004000400042F
:10357C00000400040004000400040004000400041F
:10358C00000400040004000400040004000400040F
:10359C0000040004000400040004000400040004FF
:1035AC0000040004000400040004000400040004EF
:1035BC0000040004000400040004000400040004DF
:1035CC0000040004000400040004000400040004CF
:1035DC0000040004000400040004000400040004BF
:1035EC0000040004000400040004000400040004AF
:1035FC00000400040004000400040004000400049F
:10360C00000400040004000400040004000400048E
:10361C00000400040004000400040004000400047E
:10362C000004000400040004000400030003000371
:10363C000003000300030003000300030003000366
:10364C000003000300030003000300030003000356
:10365C000003000300030003000300030003000346
:10366C000003000300030003000300030003000336
:1038DC0000020002000100010001000100010001D2
:1038EC0000010001000100010001000100010001C4
:1038FC0000010001000100010001000100010001B4
:10390C0000010001000100010001000100010001A3
:10391C000001000100010001000100010001000193
:10392C000001000100010001000100010001000183
:10393C000001000100010001000100010001000173
:10394C000001000100010001000100010001000163
:10395C000001000100010001000100010001000153
:10396C000001000100010001000100010001000143
:10397C000001000100010001000100010001000133
:10398C000001000100010001000100010001000123
:10399C000001000100010001000100010001000113
:1039AC000001000100010001000100010001000103
:1039BC0000010001000100010001000100010001F3
:1039CC0000010001000100010001000100010001E3
:1039DC0000010001000100010001000100010001D3
:1039EC0000010001000100010001000100010001C3
:1039FC0000010001000100010001000100010001B3
:103A0C0000010001000100010001000100010001A2
:103A1C000001000100010001000100010001000192
:103A2C000001000100010001000100010001000182
:0D4CCA0046044D00000000000041044C00B5
:104AD100E4900580F0900580E0FFD394024003024A
:104AE1004BDEEF25E02409F582E43404F583E0FC94
:104AF100A3E0FDE4120E457B007AC0793F784412B1
:104B01000DA3900581121094900580E025E0242FDB
:104B1100F582E43404F583E0FCA3E0FDE4120E45E4
:104B2100900581E0F8A3E0F9A3E0FAA3E0FB120C01
:104B31009A120E7E900585EEF0A3EFF0900580E0CD
:104B4100FF7E0012497E900580E0FD25E0244DF5B1
:104B510082E43404F583E0FAA3E0D39FEA9E406146
:104B6100EDFF7E0012497E900580E025E0244DF5A1
:104B710082E43404F583E0FCA3E0C39FFFEC9EFED6
:104B8100C3900586E09F900585E09E504790058083
:104B9100E0FF25E0244DF582E43404F583C083C0B1
:104BA10082E0FCA3E0FDC004C0057E0012497EC383
:104BB100D0E09FFFD0E09ED082D083F0A3EFF080C1
:104BC10013900580E025E0244DF582E43404F5835B
:0D4BD100E4F0A3F0900580E004F0024AD665
:014BDE0022B4
:103F2B00E490059FF0A3F07D077C009005A0E025B1
:103F3B00E0FF90059FE033FE90044D75F006ED1207
:103F4B0010D1EC75F006A42583F583E5822FF5825D
:103F5B00E5833EF583E0FAA3E0FB90045375F0068E
:103F6B00ED1210D1EC75F006A42583F583E5822FB5
:103F7B00F582E5833EF583EAF0A3EBF0ED1D7001CE
:103F8B001CED4C70A69005A0E025E0FF90059FE08E
:103F9B0033FE74092FF58274043EF583E0FCA3E035
:103FAB00FDE4120E457B007AC0793F7844120DA3D5
:103FBB009005A11210949005A0E025E0FF90059FBD
:103FCB00E033FE742F2FF58274043EF583E0FCA3DF
:103FDB00E0FDE4120E459005A1E0F8A3E0F9A3E0A3
:103FEB00FAA3E0FB120C9A120E7EAD07AC069005FD
:103FFB009FE0FAA3E0FB25E0FFEA33FE74532FF5B5
:10400B008274043EF583ECF0A3EDF074532FF5822C
:10401B0074043EF583E0FEA3E0D394FFEE940F40CF
:10402B0018EB25E0FFEA33FE74532FF58274043E40
:10403B00F583740FF0A374FFF090059FE0FEA3E0EF
:10404B00FF1253F8AD07AC069005A0E025E0FF90FA
:10405B00059FE033FE744D2FF58274043EF583E02B
:10406B00FAA3E0C39DEA9C500F744D2FF5827404A4
:10407B003EF583ECF0A3EDF090044CE004F0640209
:10408B006003024135124976AC06AD079005A0E0FE
:10409B0025E0FF90059FE033FE744D2FF5827404ED
:1040AB003EF583E0FEA3E0D39DEE9C40781249766B
:1040BB00AC06AD079005A0E025E0FF90059FE0332F
:1040CB00FE744D2FF58274043EF583E0FAA3E0C332
:1040DB009DFDEA9CFC74532FF58274043EF583E03E
:1040EB00FEA3E0C39DEE9C503C90059FE0FCA3E03B
:1040FB00FD25E0FFEC33FE744D2FF58274043EF585
:10410B0083C083C082E0FEA3E0FFC006C007AF05FB
:10411B00AE0412497EC3D0E09FFFD0E09ED082D088
:10412B0083F0A3EFF0E490044CF09005A0E004F0D2
:10413B00700690059FE004F0D39005A0E0940290E8
:0C414B00059FE0648094805003023F3226
:014157002245
:0849760090059FE0FEA3E0FFA5
:04497E00AB07AA06D3
:10498200EB25E0FFEA33FE744D2FF58274043EF509
:1049920083E0FEA3E0D39466EE94064036EB25E076
:1049A200FFEA33FE74032FF58274043EF583A3E01D
:1049B20025E0FF0582D5820215831582E033FE745D
:1049C2003C2FF582741A3EF583E493FC740193FD47
:1049D200024AC3EB25E0FFEA33FE744D2FF58274E1
:1049E200043EF583E0FEA3E0D39433EE9403403912
:1049F200EB25E0FFEA33FE74032FF58274043EF5E3
:104A020083A3E025E0FF0582D5820215831582E0AB
:104A120033FE743C2FF582741A3EF583E493C3137C
:104A2200FC74019313FD024AC3EB25E0FFEA33FE57
:104A3200744D2FF58274043EF583E0FEA3E0D39417
:104A420099EE9401403DEB25E0FFEA33FE74032F1B
:104A5200F58274043EF583A3E025E0FF0582D5824A
:104A62000215831582E033FE743C2FF582741A3EE0
:104A7200F583E493FE7401937802CEC313CE13D868
:104A8200F9803BEB25E0FFEA33FE74032FF58274D5
:104A9200043EF583A3E025E0FF0582D5820215835B
:104AA2001582E033FE743C2FF582741A3EF583E4DE
:104AB20093FE7401937803CEC313CE13D8F9FDACE1
:0E4AC20006ED4C7005FE7F018004AE04AF05CA
:014AD00022C3
:10596A00D3EF9DEC6480F8EE648098400122AE0487
:03597A00AF052254
:10554B00E4FDFCE4FBFAEB25E0FFEA33FE900453A9
:10555B0075F006ED1210D1EC75F006A42583F583DA
:10556B00E5822FF582E5833EF583E4F0A3F00BBBD8
:10557B0000010AEB64034A70CD0DBD00010CED6414
:04558B00084C70BF99
:01558F0022F9
:0853F8009005B2EEF0A3EFF006
:10540000E4A3F0A3F0FBFA9005B3E025E0FF9005DC
:10541000B2E033FE90045375F006EB1210D1EA753A
:10542000F006A42583F583E5822FF582E5833EF51A
:1054300083E0FCA3E0FD9005B4E0FEA3E0FF125979
:105440006A9005B4EEF0A3EFF00BBB00010AEB6429
:0C545000084A70B39005B4E0FEA3E0FF32
:01545C00222D
:104CD70046054E0000000000004605540000000095
:024CE7000000CB
:10433100E4FDFC74312DF58274053CF583E06042A7
:10434100ED25E0FFEC33FE74352FF58274043EF564
:1043510083E0FAA3E0D39400EA940440028058ED8C
:1043610025E0FFEC33FE744D2FF58274043EF58396
:10437100E0FAA3E0D394FFEA940740030244020267
:104381004443ED25E0FFEC33FE744D2FF5827404B8
:104391003EF583E0FAA3E0D394FFEA9407402B743F
:1043A100542FF58274053EF583E0FEA3E04E701AAA
:1043B100ED25E0FFEC33FE74542FF58274053EF5D4
:1043C10083E4F0A37402F0024458ED25E0FFEC33DE
:1043D100FE744D2FF58274043EF583E0FAA3E0C329
:1043E10094FFEA9407402B74542FF58274053EF52F
:1043F10083E0FEA3E064024E7018ED25E0FFEC338C
:10440100FE74542FF58274053EF583E4F0A304F0A5
:104411008045ED25E0FFEC33FE744D2FF5827404E9
:104421003EF583E0FAA3E0C394FFEA9407502874B1
:10443100542FF58274053EF583E0FEA3E064014E3E
:104441007015ED25E0FFEC33FE74542FF5827405F1
:104451003EF583E4F0A3F0ED25E0FFEC33FE745468
:104461002FF58274053EF583E0FAA3E0FB64024A6E
:10447100700E744E2FF58274053EF583740F80190A
:10448100EB64014A701AED25E0FFEC33FE744E2F08
:10449100F58274053EF5837407F0A374FFF080265E
:1044A100ED25E0FFEC33FE74542FF58274053EF5E3
:1044B10083E0FAA3E04A700E744E2FF58274053E34
:1044C100F583E4F0A3F00DBD00010CED64034C6035
:0444D100030243346B
:0144D50022C4
:100C9A00EC4D6011E8497017ED33EC3304600DE454
:100CAA00FCFFFEFD22E933E8330470F8020EEA1273
:100CBA000EB558046009E4CC248150062850090274
:100CCA000EF4284003020EF1C0E0EB4A7044B980EA
:100CDA0006D0E0FB020EE0EF4E701CBD8008EBFF71
:100CEA00EAFEE9FD80EBE98DF0A4FEE5F0020D8352
:100CFA00E9CDF9EAFEEBFFEF89F0A4FCE5F0CE8935
:100D0A00F0A42EFFE435F0CD89F0A42DFEE435F0F1
:100D1A008067EF4E7005BD80D780C3EF8BF0A4AC1F
:100D2A00F0EE8BF0A42CFCE435F0F8EF8AF0A42C5A
:100D3A00E5F038FCE433CB8DF0A42CFCE5F03BF86D
:100D4A00EE8AF0A42CFCE5F038F8E433CF89F0A45D
:100D5A002CFCE5F038CF3400CE89F0A42FFFE5F063
:100D6A003EFEE433C98DF0A42EFEE5F039CD8AF0BB
:100D7A00A42FFFE5F03EFEE43DFD33D0E0FB500733
:100D8A000BBB000F020EF4EC2CFCEF33FFEE33FE2C
:060D9A00ED33FD020ECC5A
:100DA000020EF4EC5D046005E859047003020EEADB
:100DB000120EB5580460F6EC4860F2EC7004FDFECB
:100DC000FF22C860DB2481C85009C3986002500626
:100DD000020EF19850CAF582E9294B4A7005AB82A0
:100DE000020EE075F0007C1A7880C3EF9BEE9AED5E
:100DF00099400DC3EF9BFFEE9AFEED99FDE842F09E
:100E0000DC23ACF0D0E0FFD0E0FED0E0FDAB8220F0
:100E1000E7101BEB60BAEC2CFCEF33FFEE33FEED7A
:100E200033FD020ECCE803F830E705C0F075F000A2
:100E3000EF2FFFEE33FEED33FD40B830E7C280AA5E
:100E400075F020800E75F010800575F0087D007E2D
:100E5000007F003392D530D503121070EC33401070
:100E6000EF33FFEE33FEED33FDEC33FCD5F0ED2236
:0E0E7000E5F0247EA2D513CC92E7CDCEFF2272
:100E7E00EDD2E7CD33EC3392D524814006E4FFFE6C
:100E8E00FDFC22FCE4CFCECDCC24E0501174FF80CB
:100E9E00EDC3CC13CCCD13CDCE13CECF13CF047068
:070EAE00F030D5DE021070E8
:100EB500E9D2E7C933E833F892D5EDD2E7CD33EC83
:070EC50033FC5002B2D522FC
:100ECC00EC30E7100FBF000C0EBE00080DBD000487
:100EDC000BEB6014A2D5EB13FCED92E7FD2274FF33
:100EEC00FCFDFEFF22E480F8A2D574FF13FC7D808C
:030EFC00E480EFA0
:100C1A00024158E493A3F8E493A34003F68001F257
:100C2A0008DFF48029E493A3F85407240CC8C333DB
:100C3A00C4540F4420C8834004F456800146F6DFAA
:100C4A00E4800B0102040810204080904BDFE47E10
:100C5A00019360BCA3FF543F30E509541FFEE4939F
:100C6A00A360010ECF54C025E060A840B8E493A366
:100C7A00FAE493A3F8E493A3C8C582C8CAC583CA91
:100C8A00F0A3C8C582C8CAC583CADFE9DEE780BE49
:014CE90000CA
:100EFF00E709F608DFFA8046E709F208DFFA803ED5
:100F0F0088828C83E709F0A3DFFA8032E309F608C1
:100F1F00DFFA8078E309F208DFFA807088828C8329
:100F2F00E309F0A3DFFA806489828A83E0A3F608DD
:100F3F00DFFA805889828A83E0A3F208DFFA804CB7
:100F4F0080D280FA80C680D4806980F2803380108E
:100F5F0080A680EA809A80A880DA80E280CA8033F7
:100F6F0089828A83ECFAE493A3C8C582C8CCC5836F
:100F7F00CCF0A3C8C582C8CCC583CCDFE9DEE7803F
:100F8F000D89828A83E493A3F608DFF9ECFAA9F0BE
:100F9F00EDFB2289828A83ECFAE0A3C8C582C8CC14
:100FAF00C583CCF0A3C8C582C8CCC583CCDFEADE2D
:100FBF00E880DB89828A83E493A3F208DFF980CC8F
:100FCF0088F0EF60010E4E60C388F0ED2402B40488
:100FDF000050B9F582EB2402B4040050AF2323452F
:060FEF008223900F4F73F6
:100FF500C5F0F8A3E028F0C5F0F8E5821582700287
:061005001583E038F02223
:10100B00A3F8E0C5F025F0F0E58215827002158398
:06101B00E0C838F0E822F5
:10102100E88FF0A4CC8BF0A42CFCE98EF0A42CFC6E
:101031008AF0EDA42CFCEA8EF0A4CDA8F08BF0A4EC
:101041002DCC3825F0FDE98FF0A42CCD35F0FCEB4B
:101051008EF0A4FEA9F0EB8FF0A4CFC5F02ECD3910
:0F106100FEE43CFCEAA42DCE35F0FDE43CFC227D
:10559000C2D5E830E70FB2D5E4C39BFBE49AFAE446
:1055A00099F9E498F8EC30E717B2D51255C6121104
:1055B00070E4C39BFBE49AFAE499F9E498F8800359
:1055C00012117030D50DE4C39FFFE49EFEE49DFDF3
:0455D000E49CFC2239
:0E107000C3E49FFFE49EFEE49DFDE49CFC2291
:10107E00EB9FF5F0EA9E42F0E99D42F0EC6480C8E9
:06108E0064809845F02289
:0C109400ECF0A3EDF0A3EEF0A3EFF022CF
:1010A000A8828583F0D083D0821210B71210B712B5
:1010B00010B71210B7E473E493A3C583C5F0C583DA
:1010C000C8C582C8F0A3C583C5F0C583C8C582C89A
:0110D00022FD
:0C10D100A42582F582E5F03583F583222A
:1010DD00D083D082F8E4937012740193700DA3A3A2
:1010ED0093F8740193F5828883E4737402936860B6
:0610FD00EFA3A3A380DFB6
:10110300E5092582F582E5083583F583B50804856D
:1011130082092210AF06858209F50822858209F526
:0411230008D2AF221D
:0D112700E5092582F582E5083583F5832270
:1011340075F008758200EF2FFFEE33FECD33CDCC72
:1011440033CCC58233C5829BED9AEC99E5829840F5
:101154000CF582EE9BFEED9AFDEC99FC0FD5F0D6D2
:10116400E4CEFBE4CDFAE4CCF9A88222B800C1B9FC
:101174000059BA002DEC8BF084CFCECDFCE5F0CB3A
:10118400F97818EF2FFFEE33FEED33FDEC33FCEB73
:1011940033FB10D703994004EB99FB0FD8E5E4F92E
:1011A400FA227818EF2FFFEE33FEED33FDEC33FC1B
:1011B400C933C910D7059BE99A4007EC9BFCE99A0F
:1011C400F90FD8E0E4C9FAE4CCFB2275F010EF2F54
:1011D400FFEE33FEED33FDCC33CCC833C810D70754
:1011E4009BEC9AE899400AED9BFDEC9AFCE899F88F
:0E11F4000FD5F0DAE4CDFBE4CCFAE4C8F92222
:00000001FF
